:020000040000FA
:02000000762860
:08000800E628B40000308A0074
:1000100034080739820701340234083404341034B8
:10002000403420340034B40000308A0034080F39E2
:1000300082077E3414346D345D3417345B347B3482
:100040001C347F345F343F3473346A3475346B341A
:100050002B34B400CF0000308A0034080F398207F7
:100060004028402842284E28452840284228512828
:1000700048284028422854284B2840284028572800
:10008000000008000030D00008004030D000080018
:100090004130D00008004930D00008007130D00055
:1000A00008007E30D00008000F30D000080000307B
:1000B000D0000800D201D40108005208D300D201B8
:1000C000A830D40002306F28D40803190800D40CDB
:1000D000031C0800D20A5208D30000306F285307CF
:1000E000530753075307241D013E29285A20D620C1
:1000F000B1207A288B20201896202619AA207A2849
:100100002408A3000508A40024082306A604230944
:100110002405A50408000B1D080080200B112014E5
:10012000A10B080064202030A100080020104A081C
:10013000C9004D08CC00CA0A05108510CA1CA528A4
:100140004F08860005148510080050088600051029
:100150008514080026115D28FF30860005148510DF
:10016000080000308B0085018312031307309F00C5
:100170008316031380308600FC3085006400043051
:100180008100831203138312313090008312031312
:10019000A001A501A601A701A601A801AA0110308E
:1001A000A9000030A2000430A1000800831203134C
:1001B000C601D101C7010830C80083134608840076
:0E01C0000520CF0000081320D0000800090021
:02400E00113F60
:00000001FF
